:020000020000FC
:100000000C947E020C9422000C9422000C94940018
:100010000C9422000C9422000C9422000C942200D8
:100020000C9422000C9422000C9422000C94F200F8
:100030000C9422000C9422000C9422000C942200B8
:100040000C9422001895592511005A2A1200E13EFD
:100050001300D86314003C9A150014E316007A3F8D
:10006000180098B01900A8371B00FAD51C00EE8CB8
:100070001E00FD5D2000B24A2200010101010102C3
:10008000020202020202020202040404050506063C
:10009000060808090A0A0C0C0C1011121416181A7A
:1000A0001C202224282C30343840444C525861689B
:1000B00070808A96A4B0C4D8E8FF0001020304054A
:1000C000060708090A0C0E1114181C2024282C30CD
:1000D00034383C40464A50545A616870788089945C
:1000E000A0A8B8C2D2E0F0FFFFFF0DC7C59A5778AD
:1000F000915DC1489138FC2B3322971AAD1413102F
:10010000800CB8098F07E00592048D03C302260214
:10011000AB014C010201C9009C0079005E0049005E
:1001200039002C0023001B000F930FB70F931F9370
:10013000CF93DF93C0916B00142D111F110BC1FFE2
:10014000142DD0919900109399001D0F1795072D2C
:10015000001F000BC2FF072DD0919A0000939A0058
:100160000D0F0795C0FD1027C3FF00E8100F17956E
:10017000169500E01054C0917C00CF3F61F00E193D
:100180001F0915950795CC0F10F4E00EF11ECC2336
:10019000C1F70E2D1F2DC0E0D0E0FF93F0917D0040
:1001A000FF3F49F4C02FD12F08C015950795FF0FC9
:1001B00010F4C00FD11FFF23C1F7FF91D0589298C0
:1001C0009398C5BB929AD5BB939A280C391C4A1CAC
:1001D0005B0C6C1C7D1CDF91CF911F910F910FBFA9
:1001E0000F9118950F930FB70F930CB15798789400
:1001F0001F930023F2F4102F107F103851F01039A4
:1002000041F0103B31F0103E21F010E010936000FF
:1002100090C0109360000F700395009361001091DF
:100220006D00112329F0101719F010E010936000F1
:1002300080C010916000103819F0113839F00AC0F0
:100240001395109360000093620073C01A95109389
:10025000600010C0103919F0113939F03BC0139506
:10026000109360000093620064C01A9510936000C0
:100270000023F9F40091620010916500011719F450
:100280001FEF1093650010916400011749F410915D
:1002900065001F3F31F0109364001FEF109365005D
:1002A00048C01FEF1093640010E0109388009198ED
:1002B00040C000936300109164001093650010919A
:1002C00062001093640011E010938800109389007D
:1002D000919A2FC0103B19F0113B39F011C01395C2
:1002E000109360000093620024C01A951093600080
:1002F000109162001130E9F4000F0093680019C0FA
:10030000103E19F0113E39F014C01395109360009F
:10031000009362000EC01A95109360001091620065
:10032000110F110F001F0058109366000093670013
:1003300000C01F910F910FBF0F91579A18950F93FF
:1003400002E30A95F1F70F91089527B9369A0895B7
:10035000349BFECF349A04B115B1169507951695C6
:1003600007950895222331F02F93159507952A9527
:10037000E1F72F910895442341F04F933695279547
:10038000179507954A95D1F74F910895442341F069
:100390004F93000F111F221F331F4A95D1F74F9122
:1003A000089520E0302F412F0027112706C03695F1
:1003B0002795440F10F4020F131F4423C1F708952B
:1003C00007FB07FD0195EDDF2EF4009510950894CD
:1003D000011D111D0895EF9344275527882799275C
:1003E000AA27BB27CC27DD270FC07695679530F469
:1003F000800F911FA21FB31FC41FD51F000F111F15
:10040000221F331F441F551FE62FE72B71F70A2FBA
:100410001B2F2C2F3D2FEF910895EE0FF0E0B39698
:10042000EE0FFF1FC895002D3196C895102D3196FF
:10043000C895202D3196C895302D08956F937F93E0
:10044000E72FEBDF802F912FA22FB32FE72FE3951C
:10045000E4DF081B190B2A0B3B0B8F939F93AF9381
:10046000BF93762F60E04F93B6DF4F91BF91AF916E
:100470009F918F91080F191F2A1F3B1F7F916F912A
:10048000089540E002C07C5043957C30E0F7089529
:10049000EE0FFF1FE00FF11DC8950895E00FF11D4D
:1004A000EE0FFF1FC895202D3196C895302D089569
:1004B000069506950695E4E7F0E0F0DF00271127A2
:1004C000089560E0702F703718F0703938F00CC064
:1004D00000E010E221E0E0E0F0E00BC008E011E213
:1004E00020E0ECE8FFE605C007EB1DE121E0E7E6D0
:1004F000F2EE30E070DF0E0F1F1F0895F8940FE545
:1005000012E00DBF1EBF112422243324442455249D
:1005100066247724EE24FF2400E0009388000093F3
:10052000890000937D000093910000939200009356
:10053000930000937F00009378000093790000936C
:100540007A0000936600009367000093680002E061
:1005500000937B000FEF00937C00009364000093F6
:1005600065000EE514EB26E700939B0010939C00BA
:1005700020939D0000E010E020E000939E00109387
:100580009F002093A0000FEF1FEF2FEF0093A1001B
:100590001093A2002093A30000E000939400009326
:1005A000900000936E0000936F0000936A00009328
:1005B000710004E50093690008E100936B0000E11D
:1005C00000936C0000E8009373000093740000E057
:1005D0000BBB00E00ABB0FEF08BB00E007BB00E06D
:1005E00005BB0FEF04BB0CEF02BB0EEF01BB00E03D
:1005F00003BF04E00EBD0FE103BD0AE005BD0FE03F
:1006000009B900E90AB906E806B900E809BF789413
:1006100020917F009ADE0CB51DB500938A001093DF
:100620008B000CB51DB520918A0030918B00021B08
:10063000130B05531C4008F456C00CB51DB50093B0
:100640008A0010938B0000E111E020E130E040E0EF
:1006500050E0E2B3E06FE027E2BB71DEE6B3E0FF1B
:10066000312BE1FF322BE2FF412BE3FF422BE4FF72
:10067000512B110F220F000F61F73093750040933B
:1006800076005093770000917500109176002091CC
:100690006B0030916C0000FB20F901FB35F902FB87
:1006A00036F903FB37F904FB33F905FB25F906FBA3
:1006B00026F907FB27F910FB21F911FB22F912FBA0
:1006C00023F913FB24F914FB34F915FB30F916FB5D
:1006D00031F917FB32F920936B0030936C000091D5
:1006E000770000936D0034DE20917F00C0E8C20FD8
:1006F000D0E008832395277020937F0026DE0091A9
:100700008000009369000091810000936A000091CD
:100710008200D7DE105800936E0010936F00009196
:100720008300009370000091840000937300009197
:100730008500009374000091860000937200009180
:100740008700009371006CB57DB5262F372F00917F
:100750008C0010918D00601B710B20938C003093E6
:100760008D0060938E0070938F000091690000955A
:100770009FDE60918E0070918F002DDE309195008C
:1007800040919600509197005058F0E0E09194000D
:10079000EE23A1F46091A1007091A2008091A300CA
:1007A000300F411F521F20F0361747075807C8F077
:1007B000362F472F582FE1E0F1E013C060919E00E3
:1007C00070919F008091A000301B410B520B20F0D4
:1007D00063177407850728F0362F472F582FE0E05E
:1007E000F1E0E093940050583093950040939600C8
:1007F0005093970000E010E020E0E0916C00E27878
:10080000E03849F4FF23B1F000919B0010919C0067
:1008100020919D002F7700939E0010939F002093BE
:10082000A0000095109520950093A1001093A200C0
:100830002093A30000916C000278023829F4FF2372
:1008400061F050919D0007C000916C00027019F09A
:10085000550F5FE7511D50939800509198000091FB
:100860006A0010916800011708F4012F00936A00D4
:100870001091900000917300113029F000917400E4
:10088000133009F036C014DE60918E0070918F0035
:10089000A2DD3091910040919200509193006091BF
:1008A0009000633091F0300F411F521FE0F43FEF92
:1008B0004FEF5FEF03E010916C0013FB96F0109187
:1008C0006C0014FB76F402E00CC0301B410B520BA1
:1008D00050F430E040E050E001E010916C0013FF74
:1008E00000E0009390003093910040939200509369
:1008F000930000918800002321F403E0009390000E
:1009000028C000918900002321F100E000938900B4
:1009100000917B00002319F00A9500937B0001E011
:100920000093900000E000939100009392000093E8
:10093000930000916C00007461F00FEF1FEF2FE740
:1009400000939500109396002093970001E0009388
:10095000940090E060E0709164007F3F11F498C0D3
:100960007C507136E8F701C0745F7432E8F37C5054
:1009700090917800A0917900B0917A0000917B006D
:10098000002381F50091720093DD6F937F93622FB6
:10099000732F00E010E020918E0030918F0043E033
:1009A000EADC19DD7F916F91302F412F522F90910A
:1009B0007800A0917900B0917A006A177B0738F42B
:1009C000931BA40BB50B6A177B0750F006C0930F5F
:1009D000A41FB51F6A177B0718F490E0A62FB72F46
:1009E0006A2F7B2F909378006093790070937A0040
:1009F00000916B0005FF7C5000916600109167002C
:100A000025E0B0DC202F312F020F131F020F131F20
:100A1000600F711F70937E0000916C000170C1F433
:100A20000091980010916A00212F1695203810F03F
:100A30001058120FC5DC24E095DC600F711F77237E
:100A40001AF460E070E004C07D3610F060E07CE6EF
:100A50006F937F9300916B0006FD745F12DDEEDCF7
:100A600095DC812E922EA32E7F916F9100916E00C6
:100A700010916F0024E076DC600F711F00916B0015
:100A800007FD745FFEDCDADC81DCB12EC22ED32ED2
:100A9000E0E0F0E000916C00017049F000919800F6
:100AA00010916A008DDCE12FF0E0111FFF0B009127
:100AB00093001091710075DC001FE11FF11D009182
:100AC0006C00047059F000917E00000F00561BEA84
:100AD00077DC20E017FD2FEFE10FF21F009170008F
:100AE00011270E0F1F1F112312F400E002C009F09E
:100AF0000FEF06950695EDE3F0E0CADC00927C006E
:100B000010916B00107131F400918800079500E09E
:100B1000000B09C0009193001EE243DC012FEDE5BC
:100B2000F0E0B6DC002D00937D0000919B00109159
:100B30009C0020919D0027FB30F922FB40F93427CF
:100B40003695001F111F221F00939B0010939C00DD
:060B500020939D0066CD1C
:00000001FF
